:020000000150AD
:02000B00211DB5
:02001B0041861C
:02002300410C8E
:1000500075900075B00175816F75200175892175E6
:100060008DF3D28E7598C0438780C299C298D2AB67
:10007000D2ACD29CD28CD28CD2A9D2AFD2B97530AC
:100080000175310175213F752800752964752212AB
:1000900075233475245675427875439A7544BC753A
:1000A0002500754005754501752800302FFAA20A14
:1000B000B0094008C22BC229C22A80ECE522540FA5
:1000C00045234524700BE522F454F07004C22D80C2
:1000D00002D22DE542540F45434544700BE542F4EE
:1000E00054F07004C22E8002D22EA22DB02E5007E2
:1000F000C2287540038015A22EB02D5007D2287556
:1001000040038008A22D822E400201B4D22B202869
:1001100006D229C22A01A8D22AC22901A8C0E0C059
:10012000D0C000D53013753064D5310D753103B2B0
:1001300030D5400575400CB228758CFAD520037572
:100140002006009001E9E52014C31392D52028046D
:10015000242280022442F8E630D504540F80035450
:10016000F0C493A820759000B80110D2B4C2B2A216
:100170002B92E03030643045618066B80210D2B214
:10018000C2B3A20C92E030305130444E8053B803D9
:1001900010D2B3C2B1A22992E030303E30433B804E
:1001A00040B80410D2B1C2B7A20A92E030302B306E
:1001B0004228802DB80510D2B7C2B5A20992E0300E
:1001C0003018304115801AB80610D2B5C2B4A22A30
:1001D00092E03030053040028007F590852932C228
:1001E0003100D000D0D0D0E032FC60DAF266B6BE8A
:1001F000E0FEF6EE3E9C7A9E00FD61DBF367B7BF42
:10020000E1FFF7EF3F9D7B9F8F0002C6C0E0C299E0
:10021000C298209A657401B52706E599F522806198
:100220007402B52706E599F52380567403B52706B1
:10023000E599F524804B7404B52706E599F54280CD
:10024000407405B52706E599F54380357406B52752
:1002500006E599F544802A7407B52706E599F5293E
:10026000801F7408B52708E599F521D22F801274F4
:1002700009B52704E599F5288007E599F527D0E029
:10028000320527D0E03230310132D53205D2317516
:03029000900032A9
